:0A2184000001020203030404050534
:100B8700E4F572F571F570F56FC20CC209C20BC2BC
:100B97000A121FDE1207C77E167F008E0A8F0B759B
:100BA700121675131275081675091C75101675112E
:100BB7005175161675177FEE54E07003020CCE754B
:100BC70073007574808E758F76C374A99FFF741632
:100BD7009ECF2402CF3400FEE48F6E8E6DF56CF548
:100BE7006BF56AF569F568F567AF6EAE6DAD6CAC20
:100BF7006BAB6AAA69A968A867C3120A5B5026E5A6
:100C070074256AF582E5733569F58374CDF0E56A75
:100C17002401F56AE43569F569E43568F568E43572
:100C270067F56780C4E4F56AF569F568F567AF6E3F
:100C3700AE6DAD6CAC6BAB6AAA69A968A867C31245
:100C47000A5B5031AE69AF6AE5762FF582E5753EEE
:100C5700F583E0FDE5742FF582E5733EF583EDF04E
:100C6700EF2401F56AE43EF569E43568F568E43593
:100C770067F56780B985730A85740B74002480FF54
:100C8700741634FFFEC3E5139FF513E5129EF512A4
:100C9700C3E50D9FF50DE50C9EF50CC3E50F9FF51C
:100CA7000FE50E9EF50EC3E5099FF509E5089EF5CC
:100CB70008C3E5119FF511E5109EF510C3E5179FD1
:100CC700F517E5169EF516D2E843D82090E668E0BA
:100CD7004409F090E65CE0443DF0D2AFD288D28A76
:100CE700C2A8C2AA43E808D2FB90E680E020E1054B
:100CF700D20D121D6890E680E054F7F0538EF8C2CB
:100D07000C300A051205A3C20A300C291215FE5031
:100D170024C20C121EC320091690E682E030E704B5
:100D2700E020E1EF90E682E030E604E020E0E41224
:0A0D37001DC412223F1211DA80C71A
:1005A30090E6B9E070030206541470030206D124E6
:1005B300FE700302075424FB700302064E147003FB
:1005C300020648146073146076240560030207B3BF
:1005D30012224140030207BF90E6BBE024FE6022E3
:1005E30014603324FD601114602224067048E50A68
:1005F30090E6B3F0E50B8037E51290E6B3F0E51330
:10060300802DE50C90E6B3F0E50D8023E50E90E632
:10061300B3F0E50F801990E6BAE0FF121DF0AA06C9
:10062300A9077B01EA494B600DEE90E6B3F0EF902A
:10063300E6B4F00207BF0207B812207A0207BF121E
:1006430021CD0207BF1219370207BF122068020724
:10065300BF12224340030207BF90E6B8E0247F6045
:100663001514601924027063A209E43325E0FFA284
:100673000BE4334F8041E490E740F0803F90E6BCC9
:10068300E0547EFF7E00E0D394807C0040047D0133
:1006930080027D00EC4EFEED4F2484F58274213EF2
:1006A300F583E493FF3395E0FEEF24A1FFEE34E6F8
:1006B3008F82F583E0540190E740F0E4A3F090E6E5
:1006C3008AF090E68B7402F00207BF0207B8122289
:1006D3004540030207BF90E6B8E024FE60162402FB
:1006E30060030207BF90E6BAE0B40105C20902073E
:1006F300BF0207B890E6BAE0705590E6BCE0547EBE
:10070300FF7E00E0D394807C0040047D0180027D65
:1007130000EC4EFEED4F2484F58274213EF583E414
:1007230093FF3395E0FEEF24A1FFEE34E68F82F5CD
:1007330083E054FEF090E6BCE05480131313541F7F
:10074300FFE0540F2F90E683F0E04420F0806D80AB
:1007530064122247506690E6B8E024FE6019240232
:10076300705A90E6BAE0B40104D209804F90E6BA19
:10077300E064026047803E90E6BCE0547EFF7E006A
:10078300E0D394807C0040047D0180027D00EC4E28
:10079300FEED4F2484F58274213EF583E493FF3309
:1007A30095E0FEEF24A1FFEE34E68F82F583800807
:1007B300120080500790E6A0E04401F090E6A0E02C
:0307C3004480F07F
:0107C6002210
:0300330002222F77
:04222F0053D8EF325F
:101FDE00758CE0758AC0E58954F04401F589758EDB
:081FEE0003D28CD2A9D2AF226C
:03003B000217A900
:1017A900C0E0C083C082C0D075D000C006C0073079
:1017B900C041C2C085C114052EE52E7002052DD386
:1017C900E52E94F4E52D648094814006752D00750D
:1017D9002E00AE2DAF2EEE90F800F0AE2DAF2EEF0D
:1017E900A3F0AE2DAF2E74012FF58274F83EF58368
:1017F900E514F030C105C2C185C114D007D006D0A7
:08180900D0D082D083D0E03280
:03002300021A4A74
:101A4A00C0E0C083C082C0D075D000C007309836CD
:101A5A00C298859915052CE52C7002052BD3E52C27
:101A6A00940EE52B648094804006752B00752C003B
:101A7A00AF2C90E7F0EFF0AF2C74F02FF582E4343E
:101A8A00E7F583E515F0D007D0D0D082D083D0E037
:011A9A003219
:03005B0002181177
:09181100C0E0C0D075D000C00792
:10181A00AF91530780EF6480704953917F2008414C
:10182A00E556B40120300608753230755600D201EB
:10183A00D3E53F9440E53E94065002D206753E0039
:10184A00753F00801CE556B402173007140532E5CF
:10185A0032B43603753230E532B53305755600C2F7
:03186A0007C208AA
:07186D00D007D0D0D0E0321B
:10160000120100020000004018162116000001021D
:1016100000010A0600020000004001000902350036
:1016200001010080FA0904000005FF000000070521
:101630000102400000070582020002000705810246
:1016400040000007058602000200070508020002AC
:101650000009022E0001010080FA0904000004FFC5
:10166000000000070501024000000705820240005B
:101670000007050202000200070581024000000485
:1016800003090410035100480059002D0043004392
:101690000044001603510048005900410050005317
:0B16A0000020002000200020000000BF
:100EEF0060802800030A03030202030700000002C8
:100EFF00000002000A2B0B13111511110000000046
:100F0F000000003F020A030303030307000000026F
:100F1F00000002000A2B130B111511110000000025
:100F2F000000003F032D030303030307000000022B
:100F3F00000002000A2B0B13111511110000000005
:100F4F000000003F030A0A0A0A0A0A07000000020B
:100F5F00000002000A2B130B1115111100000000E5
:100F6F000000003F60242887000000000000000000
:100F7F000000000000000000000000000000000062
:100F8F0000000000000000000000000047288080E3
:060F9F00000009CA4E002B
:10137B0090E60174CAF090E6F574FFF0902880E0D7
:10138B0090E6F3F0902881E090E6C3F0902882E09D
:10139B0090E6C1F0902883E090E6C2F0902885E0BB
:1013AB0090E6C0F0902886E090E6F4F075AF0774F5
:1013BB0028F59A7400F59B759DE4E4F59EFF90E685
:1013CB007BE090E67CF00FBF80F490E67174FFF049
:1013DB00F5B490E672E04480F043B680000000E480
:1013EB0090E6C4F000000090E6C5F0902887E090EE
:1013FB00E6C6F0902888E090E6C7F0902889E09048
:10140B00E6C8F090288AE090E6C9F090288BE0902F
:10141B00E6CAF090288CE090E6CBF090288DE09017
:0B142B00E6CCF090288EE090E6CDF0BB
:011436002293
:03004300021500A3
:0300530002150093
:10150000021FF60002203C000220260002200E00EE
:10151000021C6200021BB2000214FF0002224900FA
:1015200002224A0002224B00021BEF000217370082
:1015300002224C0002224D00021B300002199600CC
:1015400002224E000222490002224F0002225000D5
:1015500002225100022252000222530002225400B1
:1015600002225500022249000222490002224900BB
:10157000022256000222570002225800022259007D
:1015800002225A0002225B0002225C0002225D005D
:1015900002225E0002225F0002226000022261003D
:1015A000022262000222630002226400022265001D
:0815B00002226600022267001E
:101DC40090E682E030E004E020E60B90E682E0302A
:101DD400E119E030E71590E680E04401F07F147EDD
:0C1DE400001215B890E680E054FEF022DA
:101EC30090E682E044C0F090E681F0438701000091
:041ED30000000022E9
:101D6800300D0990E680E0440AF0800790E680E0B4
:101D78004408F07FDC7E051215B890E65D74FFF02C
:0F1D880090E65FF05391EF90E680E054F7F02281
:021DF000A90741
:101DF200AE16AF178F828E83A3E064037017AD0116
:101E020019ED7001228F828E83E07C002FFDEC3E63
:091E1200FEAF0580DF7E007F00B9
:011E1B0022A4
:1015B8008E7B8F7C90E600E054187012E57C240145
:1015C800FFE4357BC313F57BEF13F57C801590E6BC
:1015D80000E05418FFBF100BE57C25E0F57CE57BA7
:1015E80033F57BE57C157CAE7B7002157B4E600580
:0615F800121ED780EE2256
:101ED7007400F58690FDA57C05A3E582458370F91E
:011EE70022D8
:100FA500C18202371040C105C104045C0000000085
:100FB500015100012500044B00000000044300001E
:100FC5000000013D000156010133FF013230023EB0
:100FD5000000025400000164000239C350023000D1
:100FE50019C106C188C101C10701420001400001C4
:020FF5003600C4
:101D97008E778F789028EB7403F0E4A3F07A287B92
:101DA700EB7D027F41121FC29028EB7401F0A3E57F
:0D1DB70078F07A287BEB7D027F41021FC28D
:0514EF001214F4AF052A
:0B14F400C2B6C2B48FB1D2B4D2B6228F
:0B217900D2B6C2B48FB1D2B4D2B622ED
:0C20F500AE077FA01214F4AF060214F432
:0C210100AE077FA11214F4AF060214F424
:0C210D00AE077FA21214F4AF060214F417
:0721DD00EF44A4FF0214F41B
:0721E400EF44AEFF0214F40A
:0C211900AE077FAD1214F4AF060214F400
:0C212500AE077FA81214F4AF060214F4F9
:0C213100AE077FB01214F4AF060214F4E5
:0C213D00AE077FB11214F4AF060214F4D8
:0C214900AE077FBB1214F4AF060214F4C2
:0C215500AE077FB31214F4AF060214F4BE
:101F5000AE07AC037F8A1214F4AF061214F47F8B21
:0D1F60001214EF7F8C1214F4AF040214F47D
:0C216100AE077F871214F4AF060214F4DE
:101F6D00AE07AC037F811214F4AF061214F47F8216
:0D1F7D001214EF7F831214F4AF040214F469
:0C216D00AE077FBE1214F4AF060214F49B
:0E20B000AE05AD077F151214EFAF060214F453
:0E20BE00AE05AD077F751214EFAF060214F4E5
:041E9C00AC05AB07DF
:101EA0007D5FE4FF1220B07D3FFF1220BEFEE4FD07
:101EB000AF03122179AF041221790DBD60F20EBE7D
:021EC00040ECF4
:011EC20022FD
:061A9B008B778A7889793F
:101AA100E4F57AF57B9000011209BDFC700C7D5FB5
:101AB100FF1220B07D3FFF0220BEBCFF2DD2B675C4
:101AC1007A00757B02C2B4AB77AA78A979857B824B
:101AD100857A831209BDF5B1D2B4057BE57B70022D
:0A1AE100057AB482E0E57AB401DB77
:011AEB0022D8
:1018D600C2B77FC87E00121EF6D2B7E4FF1221E41B
:1018E6007F721220F5E4FF122101FF12210DFF1273
:1018F60021DD7F3F1221257F8E1221197F0B1221B8
:10190600317F3112213D7FF01221557B647D787F36
:1019160064121F507F3A1221497F3E12216D7F06C5
:101926001221617B7D7D507F91121F6D7F01022107
:01193600E4CC
:1007C70090E600E054E74410F000000000000090BD
:1007D700E61074A0F000000090E60B7401F090E6BC
:1007E7001274E0F0000000E490E613F000000090BF
:1007F700E61474E2F000000090E61574A0F0000023
:100807000090E6D27402F090E6047480F0000000D5
:100817007402F00000007406F00000007408F00095
:100827000000E4F000000012137B90E6187408F053
:1008370000000090E619F000000090E61AF00000B2
:100847000090E61BF0000000E490E671F075B47FBD
:1008570075A07F90E672F075B6FF75B1FF90E670F0
:10086700F075B2FF75B5FFC28CD2B012222390E6A5
:100877001074A0F000000090E611F000000090E670
:100887005EE04408F0000000E490E68DF000000010
:1008970090E65EE04404F0000000E490E7C0F090CA
:1008A700E7C4F0A3F0A3F0A3F090E7F0F090E68F91
:1008B7007440F000000090E65EE04440F000000065
:1008C7007E027F0090F800E4F0A3DFFCDEFA90E6FA
:1008D700987402F0000000E490E699F00000007EB2
:1008E700027F0090F800E4F0A3DFFCDEFA90E65EFA
:1008F700E04480F0000000E490E69CF000000090E7
:10090700E69DF00000007F9AFE12218E7527007584
:1009170028B47557017558907537107538B8755ADA
:1009270006755B2C1221D590E67AE054FEF0E4FDC3
:100937007F9012208C7F647E001215B87DFF7F4266
:1009470012208C7F647E001215B87D827F4E1220A4
:100957008C7541FF43A020E4F54990E782E541F01B
:1009670090E781E549F0122223D2087556017539BF
:1009770027753A107530007531051219F07F887E9A
:1009870013121EF61219F07F887E13121EF67FB817
:100997007E0B121EF61220E81218D67DFFE4FF1216
:1009A7001E9CD2F9C2F8E4F55190E7C0E551F04337
:0509B700A01053917F28
:0109BC002218
:0E20CC00EF2401FBE43EFA7D047F48021FA6CC
:100D4100E549C313FFC374809FF57FE549D3940040
:100D510040067541FF43A020E549700353A0DF7EA3
:100D6100287FEB1220CC9028ECE090E7C1F090288E
:100D7100EDE090E7C2F09028EB74E5F07A287BEB88
:100D81007D017F41121FC27A287BEB7D027F4112D8
:100D91001FA69028EBE0FEA3E07C002400FFEC3EC0
:100DA100FEE48F7E8E7DF57CF57B7F097E3DFDAB7C
:100DB1007EAA7DA97CA87B120A0C780D120A7FEF0E
:100DC1002490F57EEE34E8F57DED34FFF57CEC34CE
:100DD100FFF57BE4FB7A01F9F8AF7EAE7DAD7CAC2B
:100DE1007B121AEC90E7CCEFF0E4FB7A01F9F8AF53
:100DF1007EAE7DAD7CAC7B121AEC90E7CDEBF09032
:100E010028EB7450F0A3742EF07A287BEB7D027FDF
:100E110041121FC29028EB74EEF07A287BEB7D0122
:100E21007F41121FC27A287BEB7D027F41121FA6F0
:100E31009028EBE0FEA3E07C002400FFEC3EFEE402
:100E41008F7E8E7DF57CF57B9028EB7450F0A3743A
:100E51000FF07A287BEB7D027F41121FC2E47FCD28
:100E61007E55FDFCAB7EAA7DA97CA87B120A0C787D
:100E71000D120A7FEF24FEF57EEE3448F57DED3448
:100E8100FFF57CEC34FFF57BE4FB7A01F9F8AF7EEA
:100E9100AE7DAD7CAC7B121AEC90E7CEEFF0E4FBBB
:100EA1007A01F9F8AF7EAE7DAD7CAC7B121AEC9085
:100EB100E7CFEBF09028EBE541F07A287BEB7D0161
:100EC1007F21121FC29028EB7402F0A37480F07A84
:100ED100287BEB7D027F28121FC2E49028EBF0A350
:0E0EE100E57FF07A287BEB7D027F28021FC29E
:1011DA00E55F2401F55FE4355EF55EE4355DF55DB6
:1011EA00E4355CF55C0555E555700205540564AEB9
:1011FA0039AF3AE4FCFDAB5FAA5EA95DA85CC312F5
:10120A000A5B700F120D41E4F55FF55EF55DF55C62
:10121A00121F2FE564B40A1790FC00E0B411097B91
:10122A00017AFC7900121A9BE490FC00F0F56490B4
:10123A00E7C8E556F0A3E532F0E555B53128E5549F
:10124A00B53023E556601124FE600804701312209D
:10125A0052800E121F0D8009E4FFFE121D9753A043
:10126A00EFE4F554F55530003D75510190E7C0E5BE
:10127A0051F0E5B130E7032005F8121100C200E48D
:10128A00F55190E7C0E551F01219F07FB87E0B12C4
:10129A001EF61219F07F887E13121EF67F887E13BF
:0712AA00121EF61220E822DB
:0215FE00D322F6
:02223F00D322A8
:02224100D322A6
:1019370090E680E030E73A00000090E6207402F07D
:10194700000000E490E621F000000090E624740215
:10195700F0000000E490E625F000000090E6267411
:1019670002F0000000E490E627F0000000D20280B9
:1019770016000000E490E620F000000090E62174D5
:0F19870040F0000000C20290E6BAE0F552D32211
:1020680090E740E552F0E490E68AF090E68B04F0C1
:02207800D32271
:0821CD0090E6BAE0F526D322EA
:10207A0090E740E526F0E490E68AF090E68B04F0DB
:02208A00D3225F
:02224300D322A4
:02224500D322A2
:02224700D322A0
:10008000E4F577F57890E6B9E0120A93054C320072
:10009000B7B300EFB5026CB602A4BB02F6BC0357BF
:1000A000C2039FC503A9C603DEC703FDCA043FCB35
:1000B00004B3D00000059FE490E68AF090E68BF050
:1000C00090E6A0E020E1F990E68BE0F577E4F5B367
:1000D00090E60174CAF0D20000000090E60474803B
:1000E000F00000007402F0000000E4F00205A1E45A
:1000F00090E68AF090E68BF090E6A0E020E1F9909F
:10010000E68BE0F577D3943F4024E4F578744025FE
:1001100078F582E434E7F583E0FF74AB2578F58267
:10012000E43428F583EFF00578E578B440DF7F8A82
:100130007E0012218E9028ABE0FF7E001221979066
:1001400028ABE0FF7E001221A09028ABE0FF7E00EC
:100150001221A99028ACE075F004A4FFAEF01221A2
:10016000B29028ACE075F004A4FFAEF01221BB9071
:1001700028ACE075F004A4FFAEF01221C49028B0C2
:10018000E0C3940250139028CCE090E6C070057450
:100190004EF08016749CF080119028CCE090E6C060
:1001A0007005749FF08003749DF09028CEE0F54AAE
:1001B0009028CBE0F5489028CFE0F5539028D9E07F
:1001C000F547A3E0FEA3E07C002400F524EC3EF517
:1001D000239028B1E0F53BE53B7003753B01902887
:1001E000B6E0FEA3E07C002400F528EC3EF527A352
:1001F000E0FEA3E02400F558EC3EF5579028B2E06D
:10020000FEA3E02400F538EC3EF537A3E0FEA3E0C2
:100210002400F55BEC3EF55A9028BCE0FEA3E024F8
:1002200000F550EC3EF54F9028BAE0FEA3E0240024
:10023000F535EC3EF5349028E0E0540FF53DE4FD53
:100240007F9012208C9028ACE0FCA3E0FDA3E0FEA0
:10025000A3E0F54E8E4D8D4C8C4BE54EF54EE54DA5
:10026000F54DE54CF54CE4F54B0205A1E4F5787449
:10027000AB2578F582E43428F583E0FF74402578D7
:10028000F582E434E7F583EFF00578E578B440DFF4
:10029000000000E490E68AF000000090E68B7440D5
:1002A000F00205A1E490E68AF090E68BF090E6A0DB
:1002B000E020E1F990E6BCE09028EBF0E4F57890DE
:1002C000E6BEE0FFE578C39F501E74402578F582B6
:1002D000E434E7F583E0FF74EC2578F582E4342814
:1002E000F583EFF0057880D790E6BAE0C313FF906E
:1002F000E6BEE0048059E490E68AF090E68BF09048
:10030000E6A0E020E1F990E6BDE09028EBF090E671
:10031000BCE09028ECF0E4F57890E6BEE0FFE578EC
:10032000C39F501E74402578F582E434E7F583E0DE
:10033000FF74ED2578F582E43428F583EFF0057835
:1003400080D790E6BAE0C313FF90E6BEE02402FD3A
:100350007A287BEB0204AD90E74074F6F0A37413A7
:10036000F0A3740CF0A37426F0A37407F0A374EE4A
:10037000F0A37401F0A37403F0A37453F0300205EA
:10038000E4A3F0800690E74974FFF0000000E490D9
:10039000E68AF000000090E68B740AF00205A17A6C
:1003A000E77B407D047F48803DE490E68AF090E65C
:1003B0008BF090E6A0E020E1F990E68BE0F577D3B2
:1003C000940150030205A190E741E0FD7F42122015
:1003D0008C90E740E0FD7F4E12208C0205A17A2828
:1003E0007BEB7D027F41121FA6000000E490E68AAD
:1003F000F000000090E68B7404F00205A190E6BCCA
:10040000E090290BF07A297B0B7D017F50121FC2EF
:100410007A297B0B7D017F50121FC290E6BEE0FD62
:100420007AE77B407F50121FA6E490E68AF0000036
:100430000090E6BEE090E68BF00000000205A1E42B
:1004400090E68AF000000090E68BF000000090E655
:10045000A0E020E1F990E6BCE0D394075003020548
:10046000A1E09028EBF0E4F57890E6BEE0FFE578B7
:10047000C39F501E74402578F582E434E7F583E08D
:10048000FF74EC2578F582E43428F583EFF00578E5
:1004900080D790E6BEE004FD7A287BEB7F50121FE8
:1004A000C290E6BEE004FD7A287BEB7F50121FC2AB
:1004B0000205A1E490E68AF090E68BF090E6A0E0D9
:1004C00020E1F990E68BE0F578C29890E740E0C330
:1004D00094304006E0D39434400A90E740E0F46062
:1004E000030205A1E55660030205A143A01090E7B1
:1004F00040E0B4FF0AD208755601C2060205A19079
:10050000E740E0F533653270030205A1C207E0B4AD
:100510000A0375336190E740E0B40B0375336290D2
:10052000E740E0B40C0375336390E740E0B40D039B
:1005300075336490E740E0B40E0375336590E7408F
:10054000E0B40F037533667556028055E490E68A71
:10055000F090E68BF090E6A0E020E1F990E68BE0E9
:10056000F578C29890E741E070051219F08032905A
:10057000E741E0B40105121CCE802690E741E0B4CB
:100580000205121F8A801A90E741E0B40305121B8E
:1005900073800E90E741E0B4FF071220E88002D399
:0205A00022C374
:0105A2002236
:101FF600C0E0C083C082D20A5391EF90E65D7401BF
:08200600F0D082D083D0E0325B
:10202600C0E0C083C0825391EF90E65D7404F0D0A7
:0620360082D083D0E032ED
:10203C00C0E0C083C0825391EF90E65D7402F0D093
:06204C0082D083D0E032D7
:101C6200C0E0C083C08285100C85110D850D828570
:101C72000C83A37402F085080E85090F850F8285F7
:101C82000E83A37407F05391EF90E65D7410F0D0C9
:061C920082D083D0E03295
:10200E00C0E0C083C082D20C5391EF90E65D74089D
:08201E00F0D082D083D0E03243
:101BB200C0E0C083C08290E680E030E72085080C58
:101BC20085090D850D82850C83A37402F085100EA4
:101BD20085110F850F82850E83A37407F05391EF51
:0D1BE20090E65D7420F0D082D083D0E03218
:0114FF0032BA
:012249003262
:01224A003261
:01224B003260
:101BEF00C0E0C083C08290E65EE054FBF0000000CE
:101BFF0090E68F7440F0000000752B00752C00905C
:101C0F00E7F0E4F05391EF90E65FE04404F090E6E4
:0C1C1F005EE04404F0D082D083D0E032BC
:0D173700C0E0C083C082C0D075D000C007E4
:1017440090E65EE054F7F090E6A1E020E1F990E73E
:1017540080E014600F240360191460201470227553
:101764002200801D90E782E0F54190E781E0F54991
:10177400800F90E781E024FF92058005752200D256
:101784000300000090E68DE4F05391EF90E65FE0F3
:0A1794004408F090E65EE04408F01F
:0B179E00D007D0D0D082D083D0E03242
:01224C00325F
:01224D00325E
:101B3000C0E0C083C08290E65EE054BFF0000000C9
:101B400090E6987402F000000090E699E4F000003E
:101B500000F52DF52E90F800F0A3F05391EF90E6EC
:101B60005FE04440F090E65EE04440F0D082D083F5
:031B7000D0E03290
:0F199600C0E0C083C082C0D075D000C004C006BE
:1019A50090E65EE0547FF090E6A6E020E1F990E64F
:1019B5009CE0FE90E69DE07C002400F566EC3EF59B
:1019C5006500000090E69CE4F090E69DF05391EFF1
:0E19D50090E65FE04480F090E65EE04480F033
:0D19E300D006D004D0D0D082D083D0E03226
:01224E00325D
:01224F00325C
:01225000325B
:01225100325A
:012252003259
:012253003258
:012254003257
:012255003256
:012256003255
:012257003254
:012258003253
:012259003252
:01225A003251
:01225B003250
:01225C00324F
:01225D00324E
:01225E00324D
:01225F00324C
:01226000324B
:01226100324A
:012262003249
:012263003248
:012264003247
:012265003246
:012266003245
:012267003244
:0612B1008F798C7A8D7B21
:1012B70053790753B0F77F0A7E00121EF6E4F57CD8
:1012C700F57DC37402957DFFE579A807088002C301
:1012D70013D8FC30E00543800280035380FD7F0A6A
:1012E7007E00121EF64380017F0A7E00121EF6530F
:1012F70080FE7F0A7E00121EF6057DE57D700205E1
:101307007CC39403E57C6480948040B6E4F57CF567
:101317007DC37409957DFFE57BAE7AA80708800534
:10132700CEC313CE13D8F930E005438002800353B0
:1013370080FD7F0A7E00121EF64380017F0A7E0031
:10134700121EF65380FE7F0A7E00121EF6057DE50B
:101357007D7002057CC3940AE57C6480948040B16B
:1013670043B0087F0A7E00121EF653B0F77F0A7E4D
:0413770000021EF65C
:09218E00AD07AC06E4FF0212B13A
:09219700AD07AC067F040212B191
:0921A000AD07AC067F050212B187
:0921A900AD07AC067F060212B17D
:0921B200AD07AC067F010212B179
:0921BB00AD07AC067F020212B16F
:0921C400AD07AC067F030212B165
:10208C009028EBEDF0EFC313FF7A287BEB7D010278
:02209C001FC261
:0E1EE8007FC47E09121EF61222077FC47E09F7
:101EF600EF7803C333CE33CED8F9FFEF4E6007EF4A
:071F06001F70F81E80F52298
:03223300C2842240
:03223600D284222D
:03223900C283223B
:03223C00D2832228
:0622230012223C022236EB
:101F2F001222397F027E00121EF612223312223C39
:101F3F007F027E00121EF61222367F027E00021EE4
:011F4F00F69B
:10209E00E4FDFC121F2F0DBD00010CBC0EF5BD742E
:0120AE00F23F
:0120AF00220E
:0721EB00121CCE43A04022AC
:0622290053A0BF021B736D
:10143700854E46854D45854C44854B43E548B4016B
:1014470002C2B01221EBE54A60030214DB752201E8
:10145700E47FE87E03FDFCAB46AA45A944A843C345
:10146700120A5B4061E5226401705B7FDD7E031237
:1014770015B8120D41E5462418F546E54534FCF547
:1014870045E54434FFF544E54334FFF543E4FFFE07
:10149700FDE543FC7818120A6C90E7C4EFF0E4FF0F
:1014A700FEE544FDE4FC7810120A6CA3EFF0E4FFBC
:1014B700E545FEE4FDFC7808120A6CA3EFF0E5466B
:1014C700FFA3EFF0808AE522B40112AE45AF4612C2
:1014D70015B88009752201E522640160FA122229F4
:0814E700E548B40102D2B02275
:101E1C00AD07AC06D3ED9400EC9400401E0000001E
:101E2C00EE90E6D0F0000000ED90E6D1F00000005E
:0C1E3C0075BB04000000E5BB30E7FB2292
:081C2B008C7B8D7CAB07AA063F
:101C3300E4FDFCC3ED957CEC957B5022EA90E6D065
:101C4300F0000000EB90E6D1F000000075BB05004A
:0E1C53000000E5BB30E7FB0DBD00010C80D5A5
:011C61002260
:101E7300AD07AC06000000ED25E0EC3390E6D0F0B2
:101E8300000000ED25E090E6D1F000000075BB04F2
:091E9300000000E5BB30E7FB2272
:10110000C2031222151220DA7FD07E07121EF612B9
:10111000221C7FD07E07121EF612209E755102906F
:10112000E7C0E551F012143775510390E7C0E5515F
:10113000F03003030211D9E4F579F57AC3E57A9525
:1011400028E5799527500D121F2F057AE57A70EC66
:10115000057980E8E547D39400400CE547FD7C0025
:10116000AF38AE37121C2BD3E5249400E52394004E
:101170004007AF24AE23121E73E4F577F578C3E57C
:1011800078955BE577955A502C121E48E4F579F571
:101190007AC3E57A953B7480F8657998500D121FF3
:1011A0002F057AE57A70EA057980E60578E57870AA
:1011B000CD057780C9E4F579F57AC3E57A9558E5E8
:1011C000799557500D121F2F057AE57A70EC057945
:0911D00080E8AF50AE4F121E1C66
:0111D90022F3
:101E4800000000E53825E0E5373390E6D0F00000E3
:101E580000E53825E090E6D1F000000075BB0400ED
:0B1E68000000E5BB20E7033003F82278
:0721F20053A0F043A00922F5
:0721F90053A0F043A00122F6
:0722000053A0F043A00322EC
:0722070053A0F043A00222E6
:07220E0053A0F043A00622DB
:0722150053A0F043A00422D6
:0720DA007FD07E07121EF605
:0720E10053A0F043A00C2204
:07221C0053A0F043A00822CB
:0D20E80053A0F07525FF90E7CBE525F02211
:1019F0001221F27F287E0A121EF61221F97F287E1C
:101A00000A121EF61222007F287E0A121EF61222E9
:101A1000077F287E0A121EF612220E7F287E0A12E7
:101A20001EF61222157F287E0A121EF61220E17F72
:101A3000287E0A121EF612221C7F287E0A121EF62B
:0A1A4000E4F52590E7CBE525F02240
:101B730012221C1220DA7FD07E07121EF6122215C3
:101B83007FD07E07121EF612220E7FD07E07121E12
:101B9300F61222077FD07E07121EF61222007FD094
:0F1BA3007E07121EF675250390E7CBE525F0228D
:101CCE0012221C121EF21220E1121EF21222151204
:101CDE001EF212220E121EE8122200121EF2122103
:101CEE00F9121EF21221F2121EF275250190E7CBA7
:041CFE00E525F022C6
:101F8A001221F2121EF21221F9121EF2122200126C
:0C1F9A001EE875250290E7CBE525F0223B
:101874000536E536B40803E4F536E53670057F0829
:10188400FE804BE536B401067F0A7E008040E536D3
:10189400B402067F027E008035E536B403067F037A
:1018A4007E00802AE536B404067F017E00801FE5B1
:1018B40036B405067F057E008014E536B406067F3F
:1018C400047E008009E536B407077F0C7E00121DF4
:0218D400972259
:10205200C201E556600F6405600B121874053FE576
:062062003F7002053E2262
:101F0D00E556601D64056019053FE53F7002053E0D
:101F1D00121874E53F64A0453E7006F53EF53FD2BC
:021F2D00072289
:0821D500E4F51DD2E9D2AF22AE
:101C980090E678E020E6F9C2E990E678E04480F042
:101CA800EF25E090E679F090E678E030E0F990E60C
:101CB80078E04440F090E678E020E6F990E678E0B5
:061CC80030E1D6D2E92252
:101D3600A90790E678E020E6F9E51D702390E6789D
:101D4600E04480F0E925E090E679F08D18AF03A92C
:101D5600077519018A1A891BE4F51C751D01D32222
:021D6600C32296
:101D0200A90790E678E020E6F9E51D702590E678CF
:101D1200E04480F0E925E0440190E679F08D18AFC7
:101D220003A9077519018A1A891BE4F51C751D039D
:041D3200D322C322D3
:03004B00020FF8A9
:100FF800C0E0C083C082C085C084C086758600C03A
:10100800D075D000C000C001C002C003C006C00730
:1010180090E678E030E206751D060210E290E67868
:10102800E020E10CE51D64026006751D070210E270
:10103800E51D24FE605F14603624FE70030210D3A1
:1010480024FC70030210DF240860030210E2AB19CD
:10105800AA1AA91BAF1C051C8F827583001209BD33
:1010680090E679F0E51C65187070751D05806B9029
:10107800E679E0AB19AA1AA91BAE1C8E827583000B
:101088001209EA751D02E5186401704E90E678E0D1
:101098004420F08045E51824FEB51C0790E678E06A
:1010A8004420F0E51814B51C0A90E678E04440F0B6
:1010B800751D0090E679E0AB19AA1AA91BAE1C8E23
:1010C800827583001209EA051C800F90E678E044D7
:1010D80040F0751D008003751D005391DFD007D0C7
:1010E80006D003D002D001D000D0D0D086D084D092
:0810F80085D082D083D0E032E4
:101FA600121D02E51D24FA600E146006240770F364
:0C1FB600D322E4F51DD322E4F51DD32254
:101FC200121D36E51D24FA600E146006240770F314
:0C1FD200D322E4F51DD322E4F51DD32238
:030000000216AB3A
:0C16AB00787FE4F6D8FD75817F0216F20E
:1009BD00BB010CE58229F582E5833AF583E02250EF
:1009CD0006E92582F8E622BBFE06E92582F8E22239
:0D09DD00E58229F582E5833AF583E4932253
:1009EA00F8BB010DE58229F582E5833AF583E8F043
:1009FA00225006E92582C8F622BBFE05E92582C8EF
:020A0A00F222D6
:100A0C00E88FF0A4CC8BF0A42CFCE98EF0A42CFC89
:100A1C008AF0EDA42CFCEA8EF0A4CDA8F08BF0A407
:100A2C002DCC3825F0FDE98FF0A42CCD35F0FCEB66
:100A3C008EF0A4FEA9F0EB8FF0A4CFC5F02ECD392B
:0F0A4C00FEE43CFCEAA42DCE35F0FDE43CFC2298
:101AEC00C2D5E830E70FB2D5E4C39BFBE49AFAE425
:101AFC0099F9E498F8EC30E717B2D5121B22120AC8
:101B0C00F5E4C39BFBE49AFAE499F9E498F88003B2
:101B1C00120AF530D50DE4C39FFFE49EFEE49DFD53
:041B2C00E49CFC2217
:100A5B00EB9FF5F0EA9E42F0E99D42F0E89C45F0F1
:010A6B002268
:100A6C00E8600FECC313FCED13FDEE13FEEF13FF68
:030A7C00D8F1228C
:100A7F00E86010ECA2E713FCED13FDEE13FEEF138D
:040A8F00FFD8F0227A
:100A9300D083D082F8E4937012740193700DA3A3F2
:100AA30093F8740193F5828883E473740293686006
:060AB300EFA3A3A380DF06
:1016B700020B87E493A3F8E493A34003F68001F2B7
:1016C70008DFF48029E493A3F85407240CC8C33334
:1016D700C4540F4420C8834004F456800146F6DF03
:1016E700E4800B0102040810204080900EEFE47E96
:1016F700019360BCA3FF543F30E509541FFEE493F8
:10170700A360010ECF54C025E060A840B8E493A3BE
:10171700FAE493A3F8E493A3C8C582C8CAC583CAE9
:10172700F0A3C8C582C8CAC583CADFE9DEE780BEA1
:010FF70000F9
:100AB90075F008758200EF2FFFEE33FECD33CDCCF4
:100AC90033CCC58233C5829BED9AEC99E582984077
:100AD9000CF582EE9BFEED9AFDEC99FC0FD5F0D654
:100AE900E4CEFBE4CDFAE4CCF9A88222B800C1B97E
:100AF9000059BA002DEC8BF084CFCECDFCE5F0CBBC
:100B0900F97818EF2FFFEE33FEED33FDEC33FCEBF4
:100B190033FB10D703994004EB99FB0FD8E5E4F9AF
:100B2900FA227818EF2FFFEE33FEED33FDEC33FC9C
:100B3900C933C910D7059BE99A4007EC9BFCE99A90
:100B4900F90FD8E0E4C9FAE4CCFB2275F010EF2FD5
:100B5900FFEE33FEED33FDCC33CCC833C810D707D5
:100B69009BEC9AE899400AED9BFDEC9AFCE899F810
:0E0B79000FD5F0DAE4CDFBE4CCFAE4C8F922A3
:00000001FF
